:020000020000FC
:100000006DC613C0000000000000000000000000EA
:10001000000017C1A5C0EFC00000F1C00000000043
:10002000A0C000000000000000001FB64091840046
:100030005091850091FD25C097FF62E097FD63E038
:10004000609369009260C9B097FDC094C2FE03C07E
:10005000742E852E81C097FF63E097FD62E0609368
:100060006900662761606CBB9D7F40E050E0C9B0CD
:1000700097FDC094C2FC69C050931C0140931B01C2
:1000800064C097FF63E097FD62E0609369009D7F25
:1000900083FF3CC097FF62E097FD63E060936900D7
:1000A000662761606CBB92604093190150931A01FE
:1000B00060911701B0901801461B5B09B02C443BBE
:1000C00060E0560720F466276062B62E17C04836F7
:1000D00061E0560720F466276061B62E0FC0403DF0
:1000E00062E0560720F466276860B62E07C0403AE3
:1000F00065E0560718F466276460B62E4091190132
:1001000050911A014093170150931801471958094B
:1001100095FD09C094FD09C05695479593FD05C00E
:100120005695479502C0440F551F4A3F500508F0A9
:100130004AEF50911B0150931C0140931B0183FF18
:1001400004C06CE3609596239B2940E2D42E916015
:1001500083FD02C050E05DBB50E1E52E1FBE189547
:1001600018951FB6DD2011F0DA941FC040E050E072
:1001700069B197FD609562FD4AEF97FF63E097FDD7
:1001800062E060936900662761606CBB9D7F69B126
:1001900097FD609562FD5AEF451741F750E2D52E65
:1001A00040931C0140931B019160EE2011F0EA94F2
:1001B00005C051E05DBB552751605CBB90FF19C085
:1001C00050911C0140911B0195FD450F95FD4795F0
:1001D0009E7F50912A01451710F440912A01572F14
:1001E000507F552331F4242E40912801433008F0EC
:1001F000422C1FBE18951FB67E7F1FBE18951FB6D6
:1002000052E040911B01415018F000921E0109C0BC
:1002100040911E014F3F29F040911E0143954093AC
:100220001E0160912801623011F420900D013214FA
:1002300031F010F03A9401C033945A9591F71FBEF3
:1002400018951FB6601429F06092B20066241FBE94
:10025000189581FF0994452D089496FF440F10F0DE
:10026000642E40E04093B20050B78D7F652D6A3F09
:1002700070F445B1487F45B982FF09C042E04A9514
:10028000F1F74BB14B604BB9816055FF8E7F1FBEBC
:100290001895826042C02998289A82603EC02A98A8
:1002A000299A82603AC028982A9A826036C04FE024
:1002B0005B9858984A95E1F72998289A82602DC052
:1002C0004FE05B9859984A95E1F72998289A8260FF
:1002D00024C04FE059985B984A95E1F72A98299AEB
:1002E00082601BC04FE0599858984A95E1F72A98C8
:1002F000299A826012C04FE0589859984A95E1F7C0
:1003000028982A9A826009C04FE058985B984A95CD
:10031000E1F728982A9A826000C0452D40950894FC
:1003200096FF440F10F0642E40E04093B2001FBED1
:1003300018950000089521E00AC023E008C02AE0D3
:1003400006C02EE104C024E602C028EC00C014E080
:1003500000ECEFDF0A95E9F71A95D1F72A95B9F77E
:10036000089535E120E509C032E124E606C03FE00A
:1003700028E703C03CE02CE800C0599A06E90A953A
:10038000F1F70CE0289AD5DF0A95E9F7289810E4F0
:10039000032FCFDF0A95E9F71A95D1F72A9569F768
:1003A0005998089500912801033008F028C0009161
:1003B00003011091040122E00038120770F0422C72
:1003C00000920501009206010092070100920801C7
:1003D0000092090100920E0112C0232D2095221FC8
:1003E000221F322F2795317033952E7F20543009EC
:1003F000209305013093060101E000930E0108955A
:1004000000910E010015E1F0009105011091060127
:100410002091030130910401021B130B2FEF0038D0
:10042000120744F020E00F3712070CF405C00FE765
:1004300010E002C000E81FEF00930A0110930B01C7
:10044000089500910E01001581F12091070130916E
:1004500008019090090100910A0110910B01200FF1
:10046000311F911E10EF91164CF01FE091160CF405
:1004700009C02FEF3FEF1FE0912E04C020E030E0D5
:1004800010EF912E10911F014116142D18F4113008
:1004900020F005C000234AF002C0002332F420936C
:1004A00007013093080190920901089500910E010F
:1004B0000015E9F100910A01112707FD1095000FC1
:1004C000111F3091260130FD05C0343089F015959B
:1004D00007950EC0A12E902EA5949794090D1A1D74
:1004E000353031F015950795333011F01595079596
:1004F0002FEF0038120744F020E00F3712070CF4FA
:1005000005C00FE710E002C000E81FEF232D002315
:100510003AF0201B18F0213008F007C021E005C098
:100520000195200F08F001C02FEF20930C010895D2
:1005300000910E010015D9F11091080120910901D7
:100540003091270130FD05C0343089F0259517958D
:100550000EC0A22E912EA5949794190D2A1D353008
:1005600031F025951795333011F0259517950FEF3C
:100570001030200744F000E01F3F20070CF405C0B6
:100580001FEF20E002C010E02FEF00910C012223AA
:100590003AF0011B18F0013008F008C001E006C075
:1005A00010951395010F08F001C00FEF402E08952C
:1005B00007EC00937C0000917A00006800640093CF
:1005C0007A0020917A0026FDF3CF009178001091F7
:1005D000790020917A002F7720937A002EEF2093D4
:1005E000210120E02093220121E0209320012EEF21
:1005F00030E0220F331F02171307C8F020932101A8
:100600003093220122E0209320012EEF30E0922E41
:10061000A32E220F331F290D3A1D0217130738F09E
:10062000209321013093220123E02093200108959B
:1006300007EC00937C0000917A000068006400934E
:100640007A00089520917A0026FDFCCF0091780071
:100650001091790020917A002F7720937A000F3F34
:1006600023E0120778F42091210130912201021732
:10067000130740F400911F01002359F00A950093DD
:100680001F0107C000911F010F3F19F00395009350
:100690001F01401608F4042D502E089574FD02E346
:1006A00075FD00E576FD00E577FD08E2172F107F68
:1006B000112399F020912B01233061F0102F169512
:1006C00020FD01C0169522FD02C0011B03C0010FD1
:1006D00008F40FEF202E402E502E0895C8EBDBE0DB
:1006E000C0931501D09316012FEF3FE12093130122
:1006F0003093140120930F01309310013695279504
:1007000020931101309312011FEF109304010FEF9A
:10071000009303010895C0911501D091160104C002
:10072000C0910F01D0911001F894009184001091B4
:100730008500C00FD11FD0938900C09388007894A2
:100740007160209101013091020100930101109329
:100750000201021B130B2091030130910401E901F6
:10076000D695C795D695C7952C1B3D0B200F311FED
:10077000209303013093040108F008951FEF1093B4
:1007800004010FEF00930301089570FDFECFC091A7
:100790001101D0911201F89400918400109185000C
:1007A0000C0F1D1F109389000093880078947160CE
:1007B000089500910301109104011695079516956F
:1007C000079516950795169507950550100918F089
:1007D0000530100510F405E0112700931301109364
:1007E000140100930F0110931001169507950093C3
:1007F000110110931201089570FDFECFC091030105
:10080000D0910401F89400918400109185000C0FA0
:100810001D1F1093890000938800789471600895DB
:10082000789470FF089582FD01C004C080FDF8CF68
:100830007894089506E0252D209522952695277019
:100840002395F8940A95F1F710B715FDE9CF2A958D
:10085000D9F778940895789470FF089582FD01C0C7
:1008600004C080FFF8CF7894089506E0252D2095E8
:100870002295269527702395F8940A95F1F710B7DD
:1008800015FFE9CF2A95D9F778940895C0911301FF
:10089000D0911401F89400918400109185000C0F00
:1008A0001D1F10938900009388007894716008954B
:1008B00070FDFECF0895F894ABE7B1E0FD015998C3
:1008C0005B9A00917B00006400937B0003E000933F
:1008D0007C0078940895F894A2E7B1E0FD012A988D
:1008E00081FD299A00917B00006400937B0002E067
:1008F00000937C0078940895F894A9E6B1E0FD0196
:100900005B98589A00917B000F7B00937B00789452
:100910000895F894A0E6B1E0FD01299881FD289A98
:1009200000917B00006400937B0003E000937C0057
:1009300078940895F894A7E5B1E0FD015898599A84
:1009400000917B00006400937B0002E000937C0038
:1009500078940895F894A4E8B1E0FD01289881FD09
:100960002A9A00917B000F7B00937B007894089576
:10097000F89459985B9A00917B00006400937B0087
:1009800003E000937C0078940895F894AFE4B1E01C
:10099000FD012A9881FD299A00917B000064009353
:1009A0007B0002E000937C0078940895F8945B98B3
:1009B000589A00917B000F7B00937B0078940895F8
:1009C000F894ABE4B1E0FD01299881FD289A0091EB
:1009D0007B00006400937B0003E000937C0078942C
:1009E0000895F8945898599A00917B0000640093F8
:1009F0007B0002E000937C0078940895F894A3E5CE
:100A0000B1E0FD01289881FD2A9A00917B000F7BBF
:100A100000937B0078940895A9E4B1E0FD0105B14D
:100A2000087F05B90BB1047F0BB90895009115013A
:100A300010911601083E23E0120708F40895009172
:100A400015011091160105501040009315011093E7
:100A50001601089570FDFECF089504E0009326016D
:100A600004E00093270101E00093280103E00093D4
:100A70002B0190649F770895F999FECF11BDF89AE4
:100A800000B50895F999FECF00BD11BDF894FA9A0A
:100A9000F99A7894089518E020E00FEFF3DF19E059
:100AA00020E00FEFEFDF089518E020E005EAEADF2D
:100AB00019E020E00AE5E6DF089518E020E0DCDF39
:100AC000053A31F519E020E0D7DF0A3509F510E0E5
:100AD00020E0D2DF0093260111E020E0CDDF00937B
:100AE000270112E020E0C8DF0093280115E020E094
:100AF000C3DF00932B0116E020E0BEDF906401FD10
:100B00009F7B17E020E0B8DF9F7701FD906802C06F
:100B1000A4DF01D00895BFDF01E00093230100911D
:100B20002601009324012CD002E0009323010091C0
:100B300027010093240124D003E0009323010091B6
:100B40002801009324011CD004E0009323010091AC
:100B50002B010093240114D005E00093230101E050
:100B600096FF02E0009324010BD006E000932301DE
:100B700001E097FD02E00093240102D095DF089583
:100B80003091230100912401313051F0323061F075
:100B9000333071F0343081F0353091F03630A1F0DF
:100BA00010E020E06FDF14C011E020E06BDF10C028
:100BB00012E020E067DF0CC015E020E063DF08C032
:100BC00016E020E05FDF04C017E020E05BDF00C03C
:100BD000089505E0902EB9DB9A94E9F70895F8940A
:100BE000C0DBC2DBC4DBC6DBAADBBBDBBDDBBFDB40
:100BF000C1DBA5DBB6DBB8DBBADBBCDB78940895E0
:100C000090902301A0902401F894ABDBAADBA9DB30
:100C100096DB9A94D1F7AEDB92DBAA94E1F7789455
:100C20000895F894A7DB78948EDB00911B010130C6
:100C3000C0F7F89496DB83DB94DB789484DB009137
:100C40001B010A3FB0F3CBDFC4DFC3DF01E0009339
:100C5000230101E00093240100E000932501D0DF8F
:100C600005E0902E72DB00911B01013040F413DF90
:100C700087DF1ADFB4DF08E000936000AADF9A94F0
:100C800089F700912501039500932501033008F4AD
:100C9000E6CF9FDF0091240103950093240115E026
:100CA00000912301033009F413E000912301053082
:100CB00008F012E0139500912401011708F4CCCF3D
:100CC00088DF87DF0091230103950093230107301C
:100CD00008F4BFCF08E0009360007BDFF894A8958C
:100CE00004B7007004BF00916000086100936000C9
:100CF00000E00093600000E80093610000E00093D2
:100D0000610002E00EBF0FEF0DBF86DE00E005B907
:100D100007E104B900E008B900E007B900E00BB949
:100D20000BE00AB90024A0E0B0E00D92AA31E9F787
:100D3000A0E0B1E004E60D920A95E9F76DDE02E06D
:100D400005BD02E00093810001E00093B10085DE63
:100D5000B4DEFBDA06DBF5DA07DBF3DA08DBF1DA1F
:100D600001E005BB00936E0003E006BB00936F003B
:100D700001E007BB0093700000917A0002600160FF
:100D800000937A00789414DC97FF03E097FD02E06B
:100D90000093690001E00DBB002701600CBB9D7F43
:100DA000D4DACBDA00911B010130D8F7CEDA8860B3
:100DB00015E0912EC2DA90FFFECF00911B010230A8
:100DC000B8F3292F2C7330911D0120931D01231797
:100DD00079F79A9479F7877F97FF03E097FD02E010
:100DE00000936900002701600CBB9D7FF894B9DA7D
:100DF000B8DAB7DA7894A9DA00920D019EDA009198
:100E00001B010A3F08F00DCF10910D01011710F0E2
:100E100000930D01013090F7F894ACDAABDAAADA5E
:100E2000789493DA8ADA00911B010130D8F3F4DD6B
:100E300022243324442455240FEF00931F010092F1
:100E4000050100920601009207010092080100923C
:100E5000090100920E017727882700921E01009158
:100E60007A000F7700937A0000917B000064009372
:100E70007B0034DC8460706111DC6CDD5CDA1BDDCE
:100E80005ADA59DA28DD59DA37DD57DA56DA41DD30
:100E900056DA50DD52DA4FDA7F7E7062FFDB5ADDC0
:100EA0003ADC87DCC3DDD6DD06DD35DC82DCBEDD89
:100EB000D1DD11DD30DC7DDCB9DDCCDD1DDD2BDCF1
:100EC00078DCB4DDC7DD25DD26DC73DCAFDDC2DD1B
:100ED00031DD21DC6EDCAADD0091150110911601D7
:100EE000083E23E0120710F0B5DDD9CF7F7D706496
:100EF000D5DB02E000930001ADDD2CDD0CDC59DC1C
:100F000095DDA8DDD8DC07DC54DC90DDA3DDE3DC77
:100F100002DC4FDC8BDD9EDDEFDCFDDB4ADC86DDB9
:100F200099DDF7DCF8DB45DC81DD94DD03DDF3DB07
:100F300040DC7CDD009100010A9521F00093000166
:100F400089DDDBCF7F7B7068A9DB84DD03DDE8DB37
:100F50001CDC2FDC51DC01E00093000161DC70FF40
:100F600097C094DCA5DCA7DCDBDB0FDC22DC44DCF7
:100F700072DC70FF8DC08ADC9BDCADDCD1DB05DC74
:100F800018DC3ADC4DDC70FF83C080DC91DCB4DC23
:100F9000C7DBFBDB0EDC30DC5EDC70FF79C076DCAF
:100FA00087DCB7DCBDDBF1DB04DC26DC39DC70FF81
:100FB0006FC06CDC7DDCBEDCB3DBE7DBFADB1CDCAA
:100FC0004ADC70FF65C062DC73DCC4DCA9DBDDDBFE
:100FD000F0DB12DC009100010A9519F0009300018A
:100FE000BDCFF8948B7F0BB1047F0BB9599AA3E561
:100FF000B1E0FD01789414DC70FF4AC047DCD2D91F
:1010000057DCB6DC8DDBC1DBD4DBF6DB24DC70FF28
:101010003FC03CDCF5D94CDCB8DC82DBB6DBC9DB9D
:10102000EBDBFEDB70FF34C031DC0BDA41DCBEDC15
:1010300077DBABDBBEDBE0DB0EDC70FF29C026DC40
:1010400035DA36DCBDDC6CDBA0DBB3DBD5DBE8DB23
:1010500070FF1EC01BDC6CDA2BDCC3DC61DB95DBB4
:10106000A8DBCADBF8DBE4DA70FF12C00FDCEADAD7
:101070001FDCC4DC55DB89DB9CDBBEDB7F770091AA
:101080001E01013028F40091040107FD09F4B3CFDB
:0C109000C3DC22243324442455248ACEDF
:00000001FF
